:103800000C94241C0C943F1C0C943F1C0C943F1CE7
:103810000C943F1C0C943F1C0C943F1C0C943F1CBC
:103820000C943F1C0C943F1C0C943F1C0C943F1CAC
:103830000C943F1C0C943F1C0C943F1C0C943F1C9C
:103840000C943F1C0C943F1C11241FBECFE5D4E008
:10385000DEBFCDBF10E0A0E6B0E0E0E1FFE302C0D4
:1038600005900D92A436B107D9F711E0A4E6B0E0B7
:1038700001C01D92A63AB107E1F70C944B1F0C94BE
:10388000001C0F92AF93BF93CF93DF93EF93FF93FF
:10389000FC01EA01DB01C895099231961197D9F72D
:1038A000FF91EF91DF91CF91BF91AF910F9008956C
:1038B0000F921F920F93AF93BF93CF93DF93EF932A
:1038C000FF93FC01EA01DB010990199001E043D06C
:1038D00032961297C9F7FC0103E03DD005E03BD0DA
:1038E000FF91EF91DF91CF91BF91AF910F911F9019
:1038F0000F9008950F931F93EF93FF93FC0103E044
:103900002AD000E810E0E00FF11FE617F707B9F73B
:10391000FF91EF911F910F9108950F930F9222D075
:10392000082E09E018D00F900F9108950F930F9271
:10393000EF93FF9317D0FC0160935700C895802D3B
:10394000FF91EF910F900F9108950F930BD001E12C
:1039500002D00F910895E199FECF00935700E895AA
:10396000FFFF00000091570000FDFCCF089583E0A9
:1039700089B98AB188618AB908958AB1877E8AB97E
:1039800008958CB95E9BFECF5E9A08958CB19927FD
:1039900008958BB19927807890700895EF92FF92E7
:1039A0000F931F93CF93DF937B01C0E0D0E0C61746
:1039B000D70770F48C010E94C91C8823E1F30E9490
:1039C000C61CF80181938F012196CE15DF0598F36F
:1039D00081E090E0DF91CF911F910F91FF90EF90E8
:1039E0000895EF92FF920F931F93CF93DF937C0183
:1039F0008B01C0E0D0E0C017D10738F4F701819106
:103A00007F010E94C11C2196F6CF81E090E0DF91FA
:103A1000CF911F910F91FF90EF900895EF92FF9239
:103A20000F931F93CF93DF937C0100E010E0081702
:103A3000190788F4C0E0D0E000000E94C91C882368
:103A400051F4219683E0C83ED807B0F30F5F1F4FB3
:103A50000E151F0578F3DF91CF911F910F91FF9005
:103A6000EF9008950E94BD1C0E9400000895DF920F
:103A7000EF92FF920F931F93CF93DF93CDB7DEB7F3
:103A80002197DEBFCDBF8C017B011982D98061E017
:103A900070E0CE01860F971F0E94CE1C89818B316A
:103AA000B1F761E070E0C8010E94CE1C61E070E0F7
:103AB000CE01860F971F0E94CE1C89819927182F4F
:103AC000002761E070E0CE01860F971F0E94CE1C98
:103AD0008981080F111D61E070E0CE01860F971FEC
:103AE0000E94CE1C89818E30B9F4C8010196BC01B8
:103AF000C7010E94CE1C98018FEF0F3F180779F085
:103B0000F70181917F01D82621503040FFEF2F3FF0
:103B10003F07B1F7DD2019F080E090E001C0C80157
:103B20002196DEBFCDBFDF91CF911F910F91FF9006
:103B3000EF90DF900895CF92DF92FF920F931F9343
:103B4000CF93DF93182FEB016A018BE10E94C11C18
:103B50004BE1F42E812F0E94C11CF1260D2F11275D
:103B6000802F0E94C11CF0268C2F0E94C11CFC26B5
:103B70008EE00E94C11C8EE0F82621978FEFCF3F88
:103B8000D80759F0F60181916F01F8260E94C11CF7
:103B90002197FFEFCF3FDF07A9F78F2D0E94C11CB0
:103BA000DF91CF911F910F91FF90DF90CF900895FB
:103BB00099278139910559F08239910524F480398A
:103BC000910529F008C08239910519F004C082E0FE
:103BD00003C087E001C080EC99270895BF92CF927F
:103BE000DF92EF92FF920F931F93CF93DF93B82E44
:103BF0008B01FB018081C82FDD27C231D10509F47B
:103C00006DC0C331D105DCF4C330D10509F44DC01A
:103C1000C430D10544F4C130D10579F1C230D105A9
:103C200009F44AC004C1C630D10509F44AC0C630FF
:103C3000D1050CF4FCC060970CF4F9C055C0C53137
:103C4000D10509F4C8C0C631D10544F4C331D1054A
:103C500009F472C0649709F44AC0E9C0CA31D105B9
:103C600009F4D7C0CB31D10524F4669709F49AC082
:103C7000DEC06B9709F4C4C0DAC0FB01118288E092
:103C8000828381E4838386E5848382E5858389E476
:103C9000868383E5878380E580878FE5818782E35C
:103CA0008287AB016BE070E0C8C0FB0181810E949C
:103CB000D81DF801828301C0FB011182A801BE0159
:103CC000BCC0FB0183819927982F88272481820F0C
:103CD000911D9093A5018093A40107C060E070E45A
:103CE00080E090E00E947A1CF8011182A3C0FB01E1
:103CF00081819927D82FCC2782819927C82BD92B4E
:103D00001182CB0102962091A4013091A501AC0152
:103D1000BE01C901880F991F0E94411CF801EC0FD8
:103D2000FD1F12829E01369527958091A4019091E6
:103D3000A501820F931F49C0FB0181819927D82FCC
:103D4000CC2782819927C82BD92BCC24DD24CC16F3
:103D5000DD06D8F4FAE0EF2EF12CE60EF71E809186
:103D6000A4019091A501880F991FA70160E870E058
:103D70008C0D9D1D0E94581C80E890E0C80ED91E35
:103D8000E80EF91ECC16DD0650F30E94A51CF801C2
:103D90001182D695C7958091A4019091A5018C0FB1
:103DA0009D1F29C0FB0181819927D82FCC278281B3
:103DB0009927C82BD92B1182EC0FFD1F12828091FD
:103DC000A4019091A5018C0F9D1F9093A501809354
:103DD000A401239673CFFB0181819927382F2227D5
:103DE00082819927282B392B11828091A4019091EF
:103DF000A501820F931F9093A5018093A4011AC07F
:103E0000FB0111828481E82FFF27E05AFF4F808158
:103E100007C0FB01118269E081E090E00E94961CDE
:103E2000F80182831382A80164E070E006C089EC87
:103E3000F8018183A80162E070E08B2D0E949B1D38
:103E4000DF91CF911F910F91FF90EF90DF90CF9076
:103E5000BF900895CF93DF93CDB7DEB72197DEBF34
:103E6000CDBF69E081E090E00E94961C992784FF15
:103E700009C08F7E0E948D1C05C064E670E08981B8
:103E80000E94EE1D64E670E0CE0101960E94371D8F
:103E9000892B99F3F7CFCFE5D4E0DEBFCDBFCEE1DC
:103EA000F894AEEFB1E00E947F1F802D843B71F447
:103EB000AFEFB1E00E947F1F802D833C39F4ADEF5E
:103EC000B1E00E947F1F802D992781BF0E94B71CFF
:103ED0000E94C61C84E690E00E940E1D0E94C91C30
:103EE000882319F00E942A1F04C0C150C8BBCC23EC
:103EF00089F70E94321D80E090E00C94871FE199C1
:103F0000FECFBFBBAEBBE09A11960DB20895FFCFB6
:043F10001E940200F9
:0400000300003800C1
:00000001FF
